:020000040000FA
:1000000007309F00A00183168501860183128501B8
:100010008601442085174420851005103F30A50037
:10002000342044204030A5003420B830A5003420CE
:10003000C030A50034204420851005100030A500F4
:100040003C207F30A5003C200930A5003C20193021
:10005000A5003C202930A5003C204630A5003C20CE
:100060000030A5003C2033280511250886008515A1
:100070004C2085114C200034051525088600851577
:100080004C2085114C200034FF304D2864304D2821
:1000900032304D2814304D280530A100C730A20061
:1000A0000130A300A20B5528A30B5228A10B4E2808
:0200B00000341A
:02400E00183D5B
:00000001FF
